:020000020000FC
:100000000C942B000C9400000C9400000C94000045
:100010000C9400000C9400000C9400000C94000060
:100020000C9400000C9400000C94A5010C940000AA
:100030000C9482030C945B000C9400000C94C80098
:100040000C9400000C9400000C9400000C94000030
:100050000C9400000000F894EE27ECBBF1E0FBBF2D
:10006000EBBFE5BFF8E1F1BDE1BD8DE0A2E0BB274C
:10007000ED938A95E9F780E098E0A0E6ED9301978B
:10008000E9F7E4E5F0E085919591009761F0A5919D
:10009000B59105901590BF01F00105900D92019763
:1000A000E1F7FB01F0CFEFE5EDBFE8E0EEBFC0E622
:1000B000D2E00C946C02AA93EA93FA93EFB7EA9316
:1000C000AF93BF93EF93FF93AFB7AF931A930A9396
:1000D0001BB10CB1E12FEC71E1F4E0919002F0E082
:1000E000E858FD4F0083A0919002AF5FA09390026B
:1000F000A83119F4E0E0E0939002A0919202AF5F82
:10010000A0939202A83129F4E0E0E093920268946F
:1001100020F8AF91AFBFFF91EF91BF91AF910991DF
:100120001991E991EFBFF991E991A99118951A9365
:1001300088249924E0919202E03049F4E4E6F0E06A
:100140008E169F061CF0E0E019910895F3CFE09120
:100150009102F0E0E858FD4F1081A0919102AF5F4D
:10016000A0939102A83119F4E0E0E0939102F89491
:10017000E0919202E150E09392027894E12F19917C
:100180000895A0919202E0E00E94CB0CF0E0089567
:10019000AA93EA93FA93EFB7EA93AF93BF93EF93DF
:1001A000FF93AFB7AF93E091B002E030A1F0E15020
:1001B000E093B002E091AF02F0E0E956FD4FE0813C
:1001C000ECB9A091AF02AF5FA093AF02A83119F4D0
:1001D000E0E0E093AF02AF91AFBFFF91EF91BF912D
:1001E000AF91E991EFBFF991E991A9911895A0918B
:1001F000B002A831E1F35D9BFECFF894E091B0022C
:10020000E03011F45D9911C0E42DF0E0E956FD4FA6
:10021000A881A0834394E8E1E41509F44424E09123
:10022000B002EF5FE093B00202C0E881ECB97894CD
:1002300021960895E091D402F091D5023196E09391
:10024000D402F093D502E0916002E03099F0B299C7
:1002500002C00E945E0BE0917102E03011F00E943A
:100260005E0B0E94640B2CF00E945E0BE3E0E093B7
:10027000740222C00E94640B2CF00E945E0BE5E029
:10028000E0937302F30131963F01E8E5F2E0E615F1
:10029000F70530F466247724E3E0EA930E94A9048A
:1002A000A091B102AF5FA093B102A23029F4E0E0C7
:1002B000E093B1020E949A080895E0916002E03054
:1002C00011F00E94EE070E94BB070E94D907A0917F
:1002D0006302A13028F0E0916302E150E0936302F1
:1002E00008950E940E07F40131964F01E0919302A8
:1002F000F09194023196E0939302F0939402A091CE
:100300009302B09194021A9744F0E0E0E0939302D4
:10031000E09394020E945D0101C00895E09195026E
:10032000F09196023196E0939502F0939602A09197
:100330009502B09196021A973CF0E0E0E0939502A6
:10034000E09396020E941A0108950E946C0BAF93ED
:10035000BF93EF93FF93AFB7AF93E091B302EF5F1B
:10036000E093B302E13039F4ECB7E15EECBF0E94F8
:10037000F2090C940702E23059F4ECB7E15EECBFED
:10038000E1E0EA930E94E80A0E94F2090C94070255
:10039000E33039F4ECB7E15EECBF0E94F2090C9453
:1003A0000702E43059F4ECB7E05EECBFE0E0E09324
:1003B000B302EA930E94E80A0E94F209F50131961D
:1003C0005F01E8E0F0E0AE16BF062CF0AA24BB24E3
:1003D0000E94290A02C00C940702F60131966F01AF
:1003E000EAE0F0E0CE16DF0694F0CC24DD240E9493
:1003F000000BE091B202E03051F4E1E0E093B20290
:1004000078940E947101F894E0E0E093B202AF9119
:10041000AFBFFF91EF91BF91AF910E947A0B1895FA
:10042000B39958C0F894E0E0EBBBE5BB859904C0F4
:10043000DD9AA8950C941602849904C0DC9AA895BC
:100440000C941C02879904C0DF9AA8950C94220290
:10045000869904C0DE9AA8950C942802829904C05B
:10046000A89AA8950C942E02B59904C0DB9AA89579
:100470000C943402B49904C0D99AA8950C943A0209
:10048000B79904C0DA9AA8950C944002B69904C0B2
:10049000D89AA8950C944602839905C0DB9AD89AFD
:1004A000A8950C944C02B09905C0DA9AD99AA895EF
:1004B0000C945302B19905C0DB9AD89AA8950C9474
:1004C0005A02B29905C0DA9AD99AA8950C94610299
:1004D0000C94100278940895E0E0EBBBEFEFEABBD8
:1004E000E8BBE0E0E7BBE2E0E5BBE1ECE4BBE0E079
:1004F000E2BBE1BBE2E0E3BFE0E0E2BFE4E6ECBF89
:10050000E0E0EFBDEEBDEDBDECBDEBBDEABDE9BD8C
:10051000E8BDE2BDE5BDE4BDE3BDEBB7EBBFE0E0A8
:10052000E5BFE4BFE2E0E9BFE0E0EBB9E8EDEAB93E
:10053000E6E8E0BDE0E0E0BDE9E1E9B9E0E8E8B91E
:10054000E0E0E0BFE1E0E0936002E0E0E093710210
:10055000E0E0E0939502E0939602E0E0E0939302FE
:10056000E0939402CC24DD24AA24BB24882499247B
:10057000E0E0E0936102E0936202E0936302E0E076
:10058000E0936902E0936A020E94880B55240E945E
:100590008E0BE8E6F1E00E94940BE0E0E09370023D
:1005A000E0936F02E09366020E94990B6624772421
:1005B000E0E0E0937202E0937402E0937502E4E0FD
:1005C000E0937302E0E0E0937602E1E0E0937702EB
:1005D00052D6A5D39DD07894A8986297E6B3E170DF
:1005E000A0E00E94C60CE0936002A895B39B18DFC0
:1005F000E0916002E030D9F10E94C1003097B1F182
:10060000A89A0E949F0B19F062960C94ED020E942A
:10061000A70B18F0AF85AA3018F062960C94ED0283
:100620000E94B00B0E94BA0BACF40E94C20BEA0FFE
:10063000FB1FFF93EF930E949700AF91BF91EC9344
:100640000E94C20B0E94C70BE881F9813196E883B2
:10065000F983E8CFEE85E03019F062960C94ED0254
:100660000E94CE0BEBD20E945E0BA89847C00E945E
:10067000C1003097B1F1DE9A0E949F0B19F062968B
:100680000C94ED020E94A70B18F0AF85AA3018F069
:1006900062960C94ED020E94B00B0E94BA0BACF46F
:1006A0000E94C20BEA0FFB1FFF93EF930E9497007B
:1006B000AF91BF91EC930E94C20B0E94C70BE881DF
:1006C000F9813196E883F983E8CFEE85E03019F0BF
:1006D00062960C94ED020E94CE0BD0D16624772452
:1006E0000DC0E0919102A0919002EA1721F4E091EF
:1006F000AF02E41511F0DE9A01C0DE9862960C9408
:10070000ED02FFCF0E946C0BE7DE0E947A0B18957A
:10071000E0E0E093B402E093B502E0E0E093B602DB
:10072000E0E0E093B702E093B802E0E0E093B902C2
:1007300008950E94170DEF81E068EF83EE81EE5F70
:10074000EE8330E0E1E0EA930E94F700EE81EA9365
:100750000E94F700EE813E0FEF81EA930E94F700BE
:10076000EF813E0F00E010E0EE81E250D801F0E0B2
:10077000AE17BF075CF40E94D70BEA930E94F70004
:100780000E94D70B3E0F0F5F1F4FEECFE32FA0E06D
:10079000B1E0F0E00E940E0DEA1B3E2F3A930E945A
:1007A000F70048C2E0917302A881B981EC93E0910F
:1007B0006102E03069F41196E1E0EC93E09170029F
:1007C000E03029F0A881B9811196E4E0EC931CC0D7
:1007D000E33011F0E13009F412C0E23029F4A881CD
:1007E000B9811196E3E00FC0E43071F4A091B60234
:1007F000A23029F4A881B9811196E3E004C0A88150
:10080000B9811196E2E0EC93E0916502E03029F0C5
:10081000A881B9811196E5E0EC930E94DE0B0E945D
:10082000C10CA881B9811296EC930E94DE0BF07086
:10083000A881B9811396EC93E091B402F091B502CE
:100840000E94C10CA881B9811496EC93E091B40286
:10085000F091B502F070A881B9811596EC93E8810A
:10086000F9813696A0917702A083EA81EA93E7E0C6
:10087000AAD76DC01A93E0917202E03011F410E033
:1008800017C0E13011F0E23011F411E011C0E33093
:1008900011F412E00DC0E43011F0E53011F413E072
:1008A00007C0E63011F414E003C0E73009F417E0A4
:1008B000A981BA811C9311968DD712968BD7139666
:1008C00089D7149687D7159685D71696E0E0EC93CE
:1008D000EB81EA93E7E0EA93EB81FC8180D7188112
:1008E000F5C1E091B902E03011F0E0E00895E0E0F8
:1008F000E093B402E093B50276D7D99AE3E0E093AF
:100900006102E1E0089576D70895E091B902E03000
:1009100011F0E0E01CC0E881F981E0936902F093F6
:100920006A0270D7EA17FB0739F4E0916102E03000
:1009300009F060D7E1E00BC0EA81E03019F0D99A04
:10094000E2E002C0D89AE1E0E0936102E1E02396A0
:1009500008950E94150DE0E0E0937102E0937602A5
:10096000EE81E13011F0E23059F4A0917302A2302F
:1009700009F480C0E091BC02E03009F07BC01CC0EB
:10098000E33031F4E0917302E03009F473C014C035
:10099000E73091F4E0917502E43011F0E53009F4AC
:1009A00002C0E63029F4E7E0E0937502ACDF62C0F4
:1009B000E7E0E09375025EC0A091BD02A13011F0A6
:1009C0000C942C05EE81E13011F4E4E007C0E23034
:1009D00011F4E5E003C0E33011F4E6E0EE830091AA
:1009E000B7021091B8020050104024F010D70E1733
:1009F0001F0714F000E010E005D7F801EA1BFB0B1D
:100A00009F010AD7E2E0F0E00E94FB0CE217F30737
:100A10001CF402D72A1B3B0BFAD60E94BD0CDF0147
:100A2000E2E0F0E00E94FB0C2E173F071CF4EFD62B
:100A30002E0F3F1FD901E0E0F0E00E94D50C5E2FA1
:100A4000E0E0E093B9025A931A930A935EDFE1E083
:100A5000E093B902EE810CC0EE81E13011F4E1E0E7
:100A600007C0E23011F4E2E003C0E33019F4E3E040
:100A7000E09375020E941C0D279608950E94170DA1
:100A8000EF81EA3049F4AE81A23009F0D3C0AC81E5
:100A9000BD81E3E0C6D6CEC0E33051F4AE81A230D2
:100AA00009F0C8C030DFC5D6E0E0E0937002C2C0F4
:100AB000E43061F4AE81A23009F0BCC0E0E0E09324
:100AC00070020FDFAC81BD81ACD6B4C0E53099F5C2
:100AD000AE81A53009F0AEC0B3D628F0AC81BD819F
:100AE000AC91A33008F0A6C0AC81BD81AC91E1E02F
:100AF0000E94C60C1E2FAC81BD8111962C9133270C
:100B0000322F2227AC81BD8112969FD62E0F3F1F18
:100B10002050304024F07BD62E173F070CF08AC0BF
:100B2000E0E0E09370021A933A932A93EEDEAC81F0
:100B3000BD8177D67FC0E630F9F4AE81A33009F0ED
:100B400079C07ED679F0AC81BD81AC91A33051F0F3
:100B5000AC81BD81AC91A23029F0AC81BD81AC915A
:100B6000A73049F4E0E0E0937002AC81BD81EC91E4
:100B7000EA93EFDE5ED65EC0E73061F4AE81A2306C
:100B800009F058C0EF81EA93ED81FE81FA93EA9370
:100B900009DE50C0E83051F4AE81A23009F04AC0FD
:100BA000BDD5E0E0E093700244D644C0E930E1F402
:100BB000AE81A43009F03EC0AC81BD8146D6B4D52B
:100BC000F0916D02E0E0B0D5AC81BD811196EC9161
:100BD00023D6F0E0EA0FFB1FA7D5E0E0E093770211
:100BE000E093700226D626C0EB3021F5AE81A53009
:100BF00009F020C0AC81BD81AC91A03011F020D6AD
:100C0000C9F4AC81BD81EC91E093BD0211961DD673
:100C10001FD6F091B702E0E01BD6AC81BD811296E1
:100C2000EC91A091B702B091B802F0E0EA0FFB1F7F
:100C30000FD6FFD50E941E0D28960895EB81EA304D
:100C400069F4AA81A23009F041C0A881B981E3E822
:100C5000EC93EB81EA93E1E0B6D538C0E33051F490
:100C6000AA81A23009F032C0E7E0F7D5E0E0E093D6
:100C700070022CC0E630E9F4AA81A33009F026C046
:100C8000A881B981AC91A13079F0A881B981AC91EA
:100C9000A33051F0A881B981AC91A23029F0A8818C
:100CA000B981AC91A73021F4A881B981EC91D5D557
:100CB0000DC0E73059F4AA81A23009F007C0EB81DA
:100CC000EA93E981FA81FA93EA93D4DD24960895B0
:100CD0001A93E0B3E07F1E2FE12FE071A0E00E94A5
:100CE000CB0CAF81B885EC93E12FE072A0E00E94BD
:100CF000CB0CAB81BC81EC93E12FE074A0E00E94AF
:100D0000CB0CAD81BE81EC93E12FE078A0E00E9496
:100D1000CB0CA981BA81EC93188129960895E0E063
:100D2000E093BA02E093BB02E093BC02E093BD0201
:100D30000895EED4E0916F02E03051F1E0E0E093ED
:100D40006F02E1E0E093700239D5E093B402F093D2
:100D5000B502E4D4A0916102A23071F458D5A3E0A9
:100D6000B0E00E94E30CDF017ED5EA17FB071CF41C
:100D7000E4E0E09361020CC0A0916102A13041F473
:100D80004BD571D5AE17BF071CF4E4E0E0936102C8
:100D9000E0916102E13059F46FD514F476D577D53E
:100DA0007DD521F489D5E1E0E093620236C0E230DE
:100DB00051F489D56AD5AE17BF070CF08BD56ED527
:100DC00009F47AD52AC0E33079F4E0E0E0936202D6
:100DD000EFE0E0936302E0917002E03019F09ED4FE
:100DE0006BD501C070D519C0E43011F465D515C0BC
:100DF000E03099F4A0916302A13078F0E0916202B2
:100E0000E03029F039D514F440D541D506C05BD582
:100E10003CD5AE17BF070CF05DD508950E94170DA5
:100E2000E0916002E03011F00C945B07E0B3E470F5
:100E3000A0E00E94C60C0E2F003011F0DD9A01C018
:100E4000DD98E0917002E03031F4E0916F02E03023
:100E500011F4003009F40FC0E0916602EF5FE093F7
:100E60006602A0916602A33030F0E0E0E0936602F3
:100E7000E1E0E0936F02E0B3E870A0E00E94C60CEE
:100E80001E2FA091BA021A17A9F05394ECE0E515B1
:100E900080F455241093BA024CDFEBB3EF7EAE2FF3
:100EA000E091BA02E03011F0E0E101C0E0E0EA2BAD
:100EB000EBBB01C05524E6B3E07C3E2FE32FE09569
:100EC000E07C3E2F303019F0E0E0E0936402A09126
:100ED00068023A1711F40C94BA07E0916002E0300E
:100EE00009F1303029F0E0916802E32BE03C59F43D
:100EF000FAD4A53138F01DD4E7E0E0937402E1E0C4
:100F0000E09371020EC0EFD4A73458F0F4D430341B
:100F100011F4E3E001C0E1E0E0937402E1E0E0936A
:100F2000710228C0303059F0E0916802E32BE03CB8
:100F300031F0A0916102A13011F0A23049F4D3D474
:100F4000A53128F0F6D3B8D4E0E0E093700212C0E7
:100F5000CAD4A73478F0CFD4E0E0E0937002303404
:100F600029F4E1E0E0936102D89A04C0E2E0E09362
:100F70006102D99ADBC0E0916002E03009F0089587
:100F8000E0916102E03089F0E0916402EF5FE0936C
:100F90006402A0916402A43639F48ED4E0E0E093B8
:100FA0006402E1E0E093650203C0E0E0E0936402E4
:100FB0000895E6B3E095E073E093BC02E03069F099
:100FC000E0916002E03031F0E0917202E03009F02F
:100FD00098D403C0E3E0EA93BCDC08950E94170DA7
:100FE000EDB7FEB7FA93EA931F93EDB7FEB7FA9306
:100FF000EA930F93EDB7FEB7FA93EA933F93EDB7F9
:10100000FEB7FA93EA932F9363DE2F913F910F91EE
:101010001F91EBB3EF70EBBB303021F0EBB3ED7F02
:10102000E062EBBB203021F0EBB3E77FE068EBBB85
:10103000103021F0EBB3EE7FE061EBBB003021F02C
:10104000EBB3EB7FE064EBBBB19902C021E001E0C0
:10105000E0917402E73039F4E0E0E093BB02EBB3D7
:10106000E07FEBBB46C0E23059F4E1E0E093BB0225
:10107000103011F44AD403C0E0E0E09374023CC0A5
:10108000E130A9F4E0E0E093BB02103011F43DD46C
:101090000DC0003041F4EBB3E07FEBBBDA9AE2E045
:1010A000E093720203C0E0E0E093740225C0E330F5
:1010B00019F5E0E0E093BB02203089F4303039F0DC
:1010C000E7E0E0937202EBB3E07FEBBB07C0EBB36A
:1010D000E07FEBBBDB9AE4E0E09372020DC03030BE
:1010E00041F4EBB3E07FEBBBD99AE5E0E093720209
:1010F00003C0E0E0E0937402E0917402E030B1F4E8
:10110000303011F0203009F402C0E0E00DC01030A2
:1011100039F0003021F4E091BB02E03009F001C069
:1011200002C0E3E001C0E6E0E09372020E941E0DFF
:10113000249608951A9310E0E0917502E03021F4AE
:10114000E0E0E093760282C0E43081F4A091730283
:10115000A13011F0A23009F476C0E0916102E030D4
:1011600009F074C0E1E0E093750202C0E13071F46F
:10117000A0917302A13011F0A23009F464C0CDD364
:1011800010F0D2D363C0E2E2D8D360C0E53081F47E
:10119000A0917302A13011F0A23009F454C0E09183
:1011A0006102E03009F052C0E2E0E093750202C053
:1011B000E23071F4A0917302A13011F0A23009F471
:1011C00042C0ABD310F0B0D341C0E3E3B6D33EC0CE
:1011D000E63079F4A0917302A33011F0A03009F445
:1011E00032C0E0916102E03089F5E3E0E0937502FE
:1011F00002C0E33071F4A0917302A33011F0A0306B
:1012000009F421C08AD310F08FD320C0E4E495D331
:101210001DC0E730A9F4A0917302A23021F0A030E4
:1012200011F0A43009F40FC078D320F0E5E0E0938A
:10123000730209C0E5E581D3E0E0E093B90206C09E
:10124000E0E0E0937602E0E0E0937502A0917502A1
:10125000A03039F4A0917302A03011F0A23009F44B
:1012600001C003C0E0E0E093B902103019F4E1E1FD
:10127000EA93FED1ECC022D2E0E0E093CF02E0930B
:10128000D002E0E0E093D202E093D302E0E0E0930A
:10129000D102E093D602E093D7020895E881E130CD
:1012A00061F4A0917202A33021F0E091BC02E03021
:1012B00009F002C0E1E045D320C0E23061F4A09122
:1012C0007202A33021F0E091BC02E03009F002C0CC
:1012D000E2E037D312C0E33031F4E0917202E03043
:1012E00009F00FD30AC0E73039F4E0917202E03020
:1012F00011F0E7E026D301C073C072C0DFD1E091E6
:101300006002E03011F40C94D609E881E13171F10A
:10131000E23261F4A0917202A33021F0E091BC02AC
:10132000E03009F002C0E1E00CD320C0E33361F407
:10133000A0917202A33021F0E091BC02E03009F0EC
:1013400002C0E2E0FED212C0E43431F4E091720255
:10135000E03009F0D6D20AC0E53539F4E0917202E6
:10136000E03011F0E7E0EDD201C03AC0E091720246
:10137000E03011F4E3E317C0E13011F0E23011F492
:10138000E2E211C0E33011F4E1E10DC0E43011F00C
:10139000E53011F4E4E407C0E63011F4E5E503C0FC
:1013A000E73001F4E6E6EA9363D11AC0E881E2325D
:1013B00011F4E1E013C0E43411F4E3E00FC0E131D3
:1013C00011F4E2E00BC0E33311F4E0E007C0E535CF
:1013D00011F4E4E003C0E63601F4E5E0E0937302C3
:1013E000219608951A93E3B3E2701E2FE091D8027C
:1013F000E11751F4A091D902A13028F0E091D9026F
:10140000E150E093D9020CC0E091D902ED5FE09386
:10141000D902A091D902A93218F0E8E2E093D902EA
:10142000A091D902E4E10E94D00CE093D70210937E
:10143000D802E5B3EE7F0E2EE091D602A091D7023E
:10144000EA2B11F0E1E001C0E0E0E029E5BB1991F1
:101450000895AF99089578D23196E093D202F0932F
:10146000D302A091D202B091D3021A972CF0E0E0FF
:10147000E093D202E093D302E091DA02F091DB0232
:101480003196E093DA02F093DB02E091D002E03093
:10149000C1F5E091D702A091D102EA1769F1A091BC
:1014A000DA02B091DB02199730F0A091DA02B09124
:1014B000DB021C9708F018C0E091DC02EF5FE093BC
:1014C000DC02A091DC02AB3070F0E6EEE093D002DB
:1014D000E0E0E093CC02E093DC02E5E0F0E0E093B2
:1014E000D202F093D30203C0E0E0E093DC02E0E03C
:1014F000E093DA02E093DB02E091D702E093D102BD
:1015000066C0E63E29F520D2309709F522D229F0AF
:10151000E091CB02E160E093CB02A091CB02A63E2A
:1015200049F4E0E0E093CD02E093CE02E2E0E09304
:10153000D0024DC0A091CC02AF5FA093CC02A132EB
:1015400030F0E0E0E093D002E093CC0240C03FC036
:10155000E230E1F5F9D13097C1F5FBD129F0E09106
:10156000CB02E160E093CB02A091CE02AF5FA093EB
:10157000CE02A83050F1E0E0E093CE02E091CD023F
:10158000EF5FE093CD02E150F0E0E853FD4FA09112
:10159000CB02A083A091CD02A330B8F0E0E0E093AD
:1015A000D002E091C902AAE5EA27A091C802EA1791
:1015B00071F4E091CA02A5EAEA27A091C802EA17ED
:1015C00031F4E091C802EA9399DE01C008950895CC
:1015D0001A93E981E03031F0E091D602E03011F069
:1015E000E1E001C0E0E01E2FE5B3EF7BAE2F10304D
:1015F00011F0E0E401C0E0E0EA2BE5BB18815CC03B
:10160000A091CF02A13098F1A23060F0E091CF021A
:10161000E150E093CF02E0E8E093C702E0E0E0931E
:10162000C6020895E091C6029DD1E081A091C70253
:10163000EA23A0E00E94CB0CE093D602E091C7021F
:10164000E695E093C702E03091F4E0E8E093C7024A
:10165000E091C602EF5FE093C602A091C602A830F7
:1016600030F0E0E0E093CF02AF98E093D602089527
:101670001A9310E07BD1A0E0A08378D1AAEAA083DE
:1016800075D1AAEAA08372D1A6EEA0836FD1A981F9
:10169000A0836CD10F01A981EAE56BD10F01A9816B
:1016A000E5EA67D1A0E0A083AF9AE0E0E093D6023C
:1016B000E5E1E093CF02188122960895E0E0E093FF
:1016C000D402E093D5020895A091D402B091D5023E
:1016D000A935E2E0BE0708950A921A92FA926A9337
:1016E0007A938A939A93AA93BA93EA93FA93EFB769
:1016F000EA930895E991EFBFF991E991B991A99120
:101700009991899179916991F99019900990089529
:10171000E0E0E0936402E09365020895E0E0E09386
:101720006B02E0936C020895E0936D02F0936E02F9
:101730000895E0E0E0936702E09368020895E0E036
:10174000EE870E949700E98BA989A13008950E9435
:101750009700EF87AE85EA0FEE87AF85A130089539
:101760000E949700E88BAE85EA0FEE87E0E0E88301
:10177000E9830895EF85E150A881B981F0E0AE17C3
:10178000BF070895E881F981DE0112960895AE0F32
:10179000BF1FEC91AE85EA0FEE870895E889EA93C2
:1017A000E889EA93FE013496FA93EA930895F801E2
:1017B000AC81BD81AE0FBF1FEC910895E0916B022B
:1017C000F0916C020895EA93EA81FB81FA93EA931F
:1017D0000C949903E0E0EC93A981BA810895FA93FF
:1017E000EA930C949903EFEFFFEFE0936902F09313
:1017F0006A020895E0916102E093B602E4E0E093AA
:1018000061020895A0916B02B0916C020895E0917D
:101810006D02F0916E020895A0916D02B0916E027A
:101820000895EC93EF81EA93E1E0EA93EE81FF8182
:10183000D6CFEF81EA93E0E0EA93EE81FF81CFCF4C
:10184000AC81BD81AC91A1300895EC91F0E0089598
:10185000E093B702F093B8020895EA931FDDEB819D
:10186000EA93E0E0B0CFE4E0F0E00E94FB0CA0914E
:101870006902B0916A020895A1DF3197E0936B028B
:10188000F0936C02BFDF10970895C1DFBBCFEA0F62
:10189000FB1FE0936B02F0936C020895E0E0E0938D
:1018A0006202EFE0E0936302E0916902F0916A0264
:1018B000A9DFEA17FB070895E0E0E0936102EBB3CC
:1018C000EC7FEBBB08957ADF3196E0936B02F093E7
:1018D0006C020895A1DF72DFEA1BFB0BE0936B0241
:1018E000F0936C020895E0916702EF5FE093670266
:1018F000A09167020895E0E0E093670230936802E8
:1019000072CFE3E0E093740269CBEBB3E07FEBBB13
:10191000D89AE1E0E09372020895A0917602AF5F59
:10192000A0937602A0310895E5E0E0937302E0E031
:10193000E0937502E093B9020895EA9399DE11E00D
:101940000895E09374024ACBE091D202F091D30261
:101950000895E091CB02EE0FE093CB02E091D70225
:10196000E0300895F0E0E254FD4F0895E12F1F5F4D
:10197000F9CFEA27D001EC93F9CFE095F0953196B5
:101980000895EF2FFF27E7FDFFEF0895EA17E1E045
:1019900009F0EE270895EA17E1E009F4EE2708952B
:1019A000EA17E1E008F0EE270895EA17FB07E1E007
:1019B0000CF0EE270895FA9FF02DEB9FF00DEA9FB3
:1019C000E02DF10D08951CD0F6DF0EF4D6DF08955A
:1019D0000024112490E1AA0FBB1F001C111C0E1A39
:1019E0001F0A18F40E0E1F1E01C0A1609A9599F7E8
:1019F000FD01D001089504D0EBDF0EF4BEDF0895A1
:101A0000E894F7FF02C0B9DF6894B7FF06C0A0955D
:101A1000B095119600F8039400FA08951B2EBF2F7D
:101A2000F12D1A2EAE2FE12D08955A934A933A9331
:101A30002A931A930A9308955D814C813B812A81F0
:061A4000198108810895E0
:00000001FF
